:020000020000FC
:1080000000C00091780005FD0AC1F092400608E129
:10801000009353060FEF0A950023E9F700914806F5
:1080200003FFECC0E0E0F0E0079116910F3F19F478
:108030001F3F09F4E3C0F3C03BB72BBFF801209109
:10804000CA014093CA013DE930933400E89520937A
:10805000CA013BBF08953091CF0137FDFCCF3BB73C
:108060002BBFF8012091CA0113E21093CA010A0143
:10807000E8952093CA013BBF089527E402EA10E087
:108080000E94FF400E944D4178940E9487440E94C4
:10809000C144FFCF009190290F770093C304089546
:1080A00000919029002319F0025039F005C024E016
:1080B00030E007E111E218C03CC020E004EE10E21D
:1080C00050E032E0F0E0E22FEC51FF4D42A1239F5F
:1080D000F801E00DF11D428353832395203190F385
:1080E00022E22093E42030E027D001E0089554D02C
:1080F000018D0A9529F00A95A1F00A95B9F019C0E9
:10810000E0ECF0E2228930E0729615D045D0048D83
:10811000158D20A131A10217130710F400A311A39C
:10812000E4CFE0ECF0E222813381EFCFB9DF00232E
:1081300069F700E008958F010C94DA442DD0068988
:108140000F7109F0F6CF1789068907FF11C01123B7
:1081500029F0165039F0125031F0F4CF22E030E01F
:10816000B69604C0C4CF21E030E0BC96E4DFBDCFBA
:10817000155019F0145031F0E5CF0AE410E402A3D1
:1081800013A3F5CF01E010E006A317A3008D04A709
:10819000002369F30C947F41E8E7F9E20895FCDFDE
:1081A00000E000A301A302A303A304A305A306897F
:1081B00007FF05C0048D158D012B09F4BACF00917E
:1081C0008E29007621F4BADF002309F08ECF0091CA
:1081D0008E290F71013091F70E949B410023B1F766
:0281E000EDCFE1
:1081F4000C94E3440C941B4507C040E04BBFF801CA
:1082040058ED54BF2083089501E70DBF00E20EBF6F
:10821400C7E5DAE20E9461472EDFF092530600912F
:108224000020109101200A3A154511F00C94000029
:10823400F0920020F092012000E200937800F6CF43
:108244004091CA01E22FF32F0093CA010491409395
:10825400CA010895B90198018B01D2C261E0E6C256
:10826400B90198018B0108C234C262E770E2260F9B
:10827400371F0C9446476AE271E2F9CFF8940AEA90
:1082840015E5E0E0F0E2008311832091790021609C
:1082940009E731D0FFCF24E001E42DD02DE127D030
:1082A400009362002CE123D0009363001FB7F8947D
:1082B400E0E5F0E00081026000831FBF00915100FF
:1082C40001FBE6F721E000E410E001D2E6E5F0E08E
:1082D4000081097F008300E807870BEB008B008196
:1082E40004600083E0E6008101600083089530E0CB
:1082F40002E00C94224110E0EAC100E00093342132
:1083040059D00091900000932A210091910000938C
:108314002B210091920000932C2100919300009353
:108324002D210091D00101FB16F001E001C000E015
:10833400CEC09ED4AEE8B9E200918E290076003218
:10834400B9F510918F290C91569707FF15C012505B
:1083540049F01A9551F526E030E004E211E222D109
:1083640001E027C0B8D00289138920E00030120749
:10837400E1F0F80109951DC01A9521F01350A9F4F4
:1083840019D0EECF00913421002331F000E411E440
:1083940092960D931C93E4CF20E430E007E311E2BE
:1083A40001D106EE11E49496F4CF95D00FE06DD090
:1083B40000E05BC400C000E0AFD000D300E004A341
:1083C40005A302A303A30895F5DF10E084D0128B64
:1083D400138BE7E3F1E230812181203001E03007A3
:1083E40009F422C0203003E0300709F436C02130FC
:1083F400300709F44EC0203004E0300749F413D2AA
:1084040007FDFDCF40E200E06ED2E4D100E05FC0A2
:108414002330300721F401E0009334210895233000
:10842400364009F445C0A8C056D0018D128D0123F1
:1084340009F06FC0268137812030304011F424D0F8
:1084440002C01DD009F498C020E038E0A9D008E2A9
:1084540013E4B4D204A315A33CC011D019F021D065
:1084640011F412D089C0018D128D012319F00BE88B
:1084740012E402C000EC12E4028B138B2AC009E35D
:1084840011E250D00023089503E000870AE0048736
:108494000895F5DF19F005D011F4F6DF6DC083D02F
:1084A40018C0ECE1F1E22481358120303040089598
:1084B400E7E3F1E20281002349F40381013108F08A
:1084C40055C00CD000E007D0048B058B02C000938C
:1084D400352101E00895ECE1F1E20895033041F023
:1084E400023031F0043021F0053011F011E001C008
:1084F40010E01093362112E0019FF001E356FF4D86
:108504006081F1810CE111E2E62F48E050E00C9427
:108514001F4703E001D030C00093242102E0009300
:1085240028210895BD01F80150810181402FA0E365
:10853400B1E20D935C935597128130E0038120E002
:108544000D901D902D903C90139700151105220558
:10855400330510F00BD008C0041B150B0F5F1F4F21
:10856400FD01068B178B01E0DB01089508E0009301
:1085740024210AE00093282100E0089579D3ACE196
:10858400B1E2FD014689578951D01496ED91FC91D1
:1085940015970995FD012689378902D001E065C345
:1085A40008E711E205C290D0ACE1B1E2FD01068911
:1085B4001789012B39F400E018EF068B178B80E044
:1085C40098E010C0FD0106891789202F212B59F14D
:1085D400183010F4C80102C080E098E0081B190BA1
:1085E400068B178BAC0122D06481F581E62F0995A7
:1085F40008E711E207C0FD01248935892F5F3F4F49
:10860400248B358B9C010197232BE1F2F8012191F6
:108614008F012F3F81F305E0009324210DE113E442
:10862400FD01028B138BE4E00C943D4724893589CA
:1086340008E711E208954FDF248905890093782122
:108644002093792122E030E0ABDF43CF44DF04897B
:10865400158946895789202F2F73622F70E028E7E8
:1086640031E2260F371F6681F781E62F099500E076
:10867400A5D104A305A32DCFB9015CD0208127FD8A
:10868400FDCFECEC208128602083105F98018B01E2
:10869400F0DDECECF1E00081077F27CE15D0C801B6
:1086A400A22FB091CA013CD045D0008107FDFDCF77
:1086B4008AD09093C1018093C001A093C40105E3C3
:1086C40005D0B093CA01AFCF0C94314793D00C942A
:1086D400FF400E942F47C801D9012A010DC08D0116
:1086E4002CD045E08C010E94194742D08096909688
:1086F40000EE400E0FEF501EEBD079F0082F0F71F3
:1087040029F400E2401600E0500648F72D918C0150
:10871400C5DF01960FEF400EEECFE6E00C943B4729
:1087240009D0008107FDFDCF008101FF02C006E3EF
:10873400CDDF0895EFECF1E008953091CA01209166
:10874400CF0127FDFCCF23E32093CA0120E020932F
:10875400C2012093C1012093C001F80141918F010E
:108764004093C40123952032B0F33093CA01089595
:108774008A93E0DF108117FDFDCF10E045E0FDD0C6
:1087840020E02093C2011093C1010093C0018091A5
:10879400CA0105E329C09A938A93802F9091CA0154
:1087A400BFDF41D007FDFDCF0ED00093C101009380
:1087B400C0018093C40103950032C8F39093CA01A9
:1087C40089919991089503E30093CA0100E000930D
:1087D400C20108958A930FEFDEDFACDF008107FD4D
:1087E400FDCF8091CA0100E305D071DF8093CA01F7
:1087F400899108950093CA0121E00BEC11E00895DA
:10880400BC01C80110D007FDFDCF042F052B49F092
:10881400FC010491F90101939F01019641505040DC
:10882400F4CFCB0108950091CF0108950E942A4707
:10883400229739012A01A62ED801912F80E006C083
:108844002091CF0127FDFCCF45E24DD041D0E1F18D
:108854009924E9DF07FDFDCF00E8802EAA2061F00E
:10886400FC01059114910883198308810F3F1F4F60
:1088740031F09924939403C00FEF0883098328D01F
:1088840071F0A817B90721F426D0088321D039F054
:10889400FC013196AE17BF0711F41DD0098348813E
:1088A40059818C0120E030E00E942B4002968A948A
:1088B400A9F69C013A959920890111F62091CF01DE
:1088C40027FDFCCF44E2C1CF2296EBE00C9436475F
:1088D400042D052908950FEF400E501E1196F30143
:1088E40001913F01089520E030E00C941C402AE1FE
:1088F40007D00093FA042BE103D00093FB040895FE
:10890400F6DC0F3F09F40FE108950E94324700E0BE
:108914000093600023E004E4EEDC68D2006400838A
:1089240001E0009360000FB7F894A02F20E030E03E
:10893400890122D0F801E858F64D35832395223079
:10894400B8F3D5DF0091C0040093C0044FD200688F
:10895400008300810061008388E799E20496E6ECD5
:1089640080839183E0EC2FD10FEF0583E8ECBBDC2F
:10897400AFBFE3E00C943E4743E00C9413471FB7AA
:10898400F89400E437D200E235D2E1ECF4E0ABDC59
:10899400E9EC008102600083E8EC0081006400835C
:1089A400E9ECA1DCE8EC0081006800831FBF0895B6
:1089B40005D0068F178F20A331A30895E8E7F9E2C5
:1089C400089562D00091CB0407FF02C000E82EC0D6
:1089D400F6D1002361F5EBEC0AD204FF1EC000E1DE
:1089E40009D200E00093A42901E010E000939E293D
:1089F40010939F2900E00093C30420E430E057D093
:108A040020E430E010E000E852D007EA19E20093D5
:108A140080291093812928D10AC0008106FF02C051
:108A240000E404C0008105FF02C000E2E3D11CD0D1
:108A340018952AD0E2D10023B1F402E00093CC04CB
:108A44000091C50432D0F801008105FF06C02DD085
:108A540020E2F80126930FD106C000E827D020E2D7
:108A6400F8012693B3D0E3CF8FBF099119912991CF
:108A74003991499159916991799109901990299065
:108A84003990E991F991B4CE8A93FA93EA933A92A0
:108A94002A921A920A927A936A935A934A933A932D
:108AA4002A931A930A938FB7089500E01AC08A9301
:108AB4002051304041F02051304039F020523040B4
:108AC40031F080E005C081E003C082E001C083E0B2
:108AD400EDDF20E0F801218326E020838064818398
:108AE40087CE6CE779E2202F2F70220F402F440F9E
:108AF40000E010E0001F020F3FDF060F171F08956C
:108B04009D01E8EC74D10F7D008300810F7D00830B
:108B14003FD102E00593A6E8B9E200E010E00D932E
:108B24000C93539600E2069300E406933BD106931C
:108B340000E406931D931D931D931C9315971D9399
:108B44001C9311A7D90108950CD1002331F00330EF
:108B540011F0043009F429D187D030DF0681178160
:108B6400083050E0104039F548E027EA39E20EE8D1
:108B740019E27FDBE8ECF4E026D025D00E94CF4058
:108B8400002309F4F1C01ADF068907FF0BC000A116
:108B94000F7311F401E001C000E006A70ED002E05B
:108BA40005A714C0048D158D012B09F405C005D04B
:108BB40001E005A7F3D00895E3C000E000A701A7F2
:108BC40002A703A70895008100628FCB51D0C7D0BC
:108BD400033011F448D046C0FD0120A131A142A5C3
:108BE40053A58901041B150B402F412B21F506A524
:108BF400002311F4D0D036C000A511A5020F131F15
:108C0400248D358D0217130728F089D019F00995A2
:108C1400002339F400E00093A629FD0106870787A5
:108C24001FC070D020A111A1022F2F7311F421E0D5
:108C340001C020E026A7013420E0120710F000E470
:108C440010E006871787268D378D42A553A5240F7C
:108C5400351F208B318B9A01200F311F22A733A798
:108C640097D09DD002C0A1D04BCFA991B9910895BE
:108C7400BA93AA93089528DD72D0043011F4F3DF77
:108C840040C0FD018681978162A573A520A131A111
:108C94008B01080F191F2017310718F4C901861B0F
:108CA400970BAC0127EA39E2068D178D060F171FC3
:108CB400E0DAFD0102A513A5080F191F02A713A7E7
:108CC4008034904031F426D0448D558D24173507D7
:108CD40060F000A311A394966FD029F009950023A6
:108CE40011F442D00EC04CD00CC020A131A12017E9
:108CF400310731F414D0A9F30995002391F302D07C
:108D04004DD091CCFD0102A513A504D020A731A715
:108D140000E056CF20A531A5200F311F0895949669
:108D2400ED91FC91959700E0E030F00708950091F3
:108D34007C2905FD07C015D0013009F43DCF04306E
:108D440009F415D008950091842905FD07C009D0C0
:108D5400023009F420C0033009F409D00895A8E7CB
:108D6400B9E20091A529089505E00093A529E5E855
:108D7400F9E204E00593EDE7F9E204E005930895D0
:108D84001DDE03E005A700E00687078701D007C0C2
:108D9400E4E8F9E2089504E00093A52903D002E091
:108DA40006930895ECE7F9E2089562DFAAE9B9E2CF
:108DB40003D009F0099559CFED91FC91B4CFEBECB8
:108DC40016D002FF07C0F093CA040091842906FD5F
:108DD400AEDF7FCB008101FF08C002E00BD0009121
:108DE4007C2906FFF6CFAFDFF4CFC6CBE0ECF4E08E
:108DF400008108950093CA0408950091CC0400FFF3
:108E0400BBCB01E00093CC04CDDF00E80693C0DFC8
:108E140000E8069301E0EEDFC5DF00E1069394DE8F
:108E240058CB4A951AF0000F111FFBCF08954A95AD
:108E34001AF016950795FBCF0895AF93BF93D80109
:108E440001900D9241505040D9F7BF91AF910895D0
:108E5400AA929A928A927A926A925A924A92BA936D
:108E6400AA939A938A930895AA84998488847F8084
:108E74006E805D804C80BB81AA8199818881F0E0FD
:108E8400EC0FFD1FEF010895BD01D801F90104C0E5
:108E940021912D9341505040242F252BC9F7DB01FC
:108EA400089520E006D0E9F70895259102D0E9F766
:108EB40008952D9301501040202F212B089586EF03
:108EC4009EE8FC0105911491FC013296A591B491A0
:108ED400FC01349625913491422F432B19F0F9016A
:108EE400E4DF01C0DEDF06961FE88230910748F315
:108EF4000895CB081C210000A9007220028F0300F2
:108F040000008000002C4130410004000032413652
:108F1400410300000037410000040000003D41000F
:108F240000000000000000000075207D20952095C1
:108F34002085208D2095209520952095209520959D
:108F44002095209520952095209520000902120057
:108F5400010100C0320904000000FF0000001201FA
:108F6400000200000040EB03E42F030000020001B4
:108F740000030000000000000000000000000000EA
:108F840000000000000000000000000000000000DD
:108F94000000444655204154584D45474133324121
:078FA4003455000403090429
:040000030000800079
:00000001FF
